:10010200120100020000004005168080000001027A
:020112000001EA
:0A0116000A0600020000004001008C
:100122000902270001010080320904000003FF00D8
:10013200000007058102400000070582020002005C
:07014200070588020002001E
:10014A000902270001010080320904000003FF00B0
:10015A0000000705810240000007058202400000F6
:07016A0007058802400000B8
:100172001403000000000000000000000000000066
:10018200000000000C0341004300430045005300FF
:100192001E035700410054004300480044004F0032
:1001A2004700000000000000000000000000000006
:0A3144000001020203030404050564
:10008000EC4EFEED4F2444F58274313EF583E4934B
:10009000FF3395E0FEEF24A1FFEE34E68F82F58377
:1000A0002290E6BCE0547EFF7E00E0D394807C008A
:1000B00022F0E52C2401F52CE4352BF52BE4352A30
:1000C000F52AE43529F52922AF30AE2FAD2EAC2D1F
:1000D000AB2CAA2BA92AA829C3020807E536252C90
:0900E000F582E535352BF583228C
:10194800E4F534F533F532F531C23CC239C23BC255
:101958003A122B067E017F028E0A8F0B75120175D3
:10196800131675080175092275100175114A751449
:1019780001751572EE54E07003021A34753500755E
:1019880036808E378F38C374B09FFF74019ECF2482
:1019980002CF3400FEE48F308E2FF52EF52DF52C76
:1019A800F52BF52AF5291200C8500A1200DC74CD6F
:1019B8001200B180F1E4F52CF52BF52AF529120077
:1019C800C85017E538252CF582E537352BF583E027
:1019D800FF1200DCEF1200B180E485350A85360B72
:1019E80074022480FF740134FFFEC3E5139FF513CE
:1019F800E5129EF512C3E50D9FF50DE50C9EF50C5D
:101A0800C3E50F9FF50FE50E9EF50EC3E5099FF59B
:101A180009E5089EF508C3E5119FF511E5109EF547
:101A280010C3E5159FF515E5149EF514D2E843D8C3
:101A38002090E668E04409F090E65CE0443DF0D28E
:101A4800AFD241122C9C90E680E054F7F0538EF808
:101A5800C23C303A05121307C23A303C291231A071
:101A68005024C23C122D9B20391690E682E030E7C4
:101A780004E020E1EF90E682E030E604E020E0E4D4
:0B1A8800122CCB1231A212218280C769
:1013070090E6B9E070030213B814700302140C24BA
:10131700FE700302146624FB70030213B2147003F9
:101327000213AC1460731460762405600302149DE5
:1013370012319840030214A990E6BBE024FE602214
:1013470014603324FD601114602224067048E50AF6
:1013570090E6B3F0E50B8037E51290E6B3F0E513BE
:10136700802DE50C90E6B3F0E50D8023E50E90E6C1
:10137700B3F0E50F801990E6BAE0FF122CF7AA0642
:10138700A9077B01EA494B600DEE90E6B3F0EF90B9
:10139700E6B4F00214A90214A212316C0214A912C5
:1013A70031620214A9122EAD0214A9123158021487
:1013B700A912319A40030214A990E6B8E0247F608D
:1013C700151460192402703AA239E43325E0FFA20C
:1013D7003BE4334F8018E490E740F080161200A1F9
:1013E70040047D0180027D00120080E0540190E7F7
:1013F70040F0E4A3F090E68AF090E68B7402F002E6
:1014070014A90214A212319C40030214A990E6B851
:10141700E024FE6016240260030214A990E6BAE0F5
:10142700B40105C2390214A90214A290E6BAE07009
:101437002C1200A140047D0180027D00120080E093
:1014470054FEF090E6BCE05480131313541FFFE0E2
:10145700540F2F90E683F0E04420F08045803C1243
:10146700319E503E90E6B8E024FE601A24027032A6
:1014770090E6BAE0B40104D239802790E6BAE0B426
:101487000202801E80151200A140047D0180027DAA
:10149700001200808008121FB8500790E6A0E044B1
:0A14A70001F090E6A0E04480F0227E
:0300330002319106
:0431910053D8EF32EE
:102E4E00E4FBFA903FB4E0FCA3E0FDA3E0FEA3E0B8
:102E5E00FF0202ADE4FFFE7D807C471201B5020445
:012E6E000162
:10236B008F428E418D408C3FE4FFFEFDFCAB42AAB9
:10237B0041A940A83F74E012034C7003C28E22E5C2
:10238B0089540F4410F589538EEF79407841122E02
:10239B004EAB42AA41A940A83F1202AD8F468E45D3
:1023AB008D448C43AB46AA45A944A843122E628E9A
:1023BB00778F78C28EEFF58BE577F58DD2ABD28E1A
:0123CB0022EF
:10277D008F428E418D408C3F79807840122E4EAB2A
:10278D0042AA41A940A83F1202ADAB07AA06A9056E
:10279D00A804122E62AD07AC06E4F5C8438E20AF37
:1027AD0004ECF5CB8FCDAF05EDF5CA8FCCD2BDD2F4
:0427BD00ADD2CA22AD
:03001B00022FBAF7
:102FBA00C0E0C0D0E578F58BE577F58DA291B392A4
:062FCA0091D0D0D0E032EE
:03002B00022804A4
:10280400C0E0C0F0C083C082C085C084C086758625
:1028140000C0D075D000C000C004C005C006C00709
:102824001229B9C2CFD007D006D005D004D000D029
:10283400D0D086D084D085D082D083D0F0D0E0327E
:102D4C00504349652D5744472D43534D4100504343
:102D5C0049652D5744472D43534D00504349652D2C
:082D6C005744472D78787800E8
:102F8C00423F000000C13FC13D0167FFC13E0163EC
:042F9C000001646468
:10164500A3E0FFAB430545E545AA4422E0FEA3E040
:10165500FDAC3F053F74402CF582E434E7F583ED9E
:10166500F0EEFFAE3F053F74402EF582E434E7F51A
:101675008322F0E5801313543F2214F9EF0207701B
:10168500EE75F003A4243EF582E4343FF583229001
:10169500E6BDE0FE90E6BCE02400FDEC3EFC90E6F5
:1016A500BFE0FE90E6BEE07A002400FBEA3EFA22A7
:1016B500E090E740F0E490E68AF090E68B22EE7544
:1016C500F003A42440F582E4343FF58322253AF55E
:1016D5003AE53D3539F539C3E53C953EF53CE53B05
:1016E500953DF53B227586005391EF90E65D22749A
:1016F500402540F58274E7353FF58322E0FFAB4393
:101705000545E545AA4422AD3E7AE779407F40ABE1
:10171500072290E6BBE0FE90E6BAE07C002400FFDD
:10172500EC3EFE22C3E540953EE53F953D22E49023
:10173500E68AF090E6BEE090E68BF02275F003A411
:10174500243FF582E4343FF5832290E68AE53EF0B6
:1017550090E68BE53DF022E53A2540F582E5393501
:101765003FF583227DFA7F007E007C4422740025AC
:1017750039F9EE34FCFA7B0122F582E4343FF58336
:1017850022F0A37401F0A3F0E4A3F022903F15E04A
:10179500FE903F14E0FD22850D82850C83A3740223
:1017A500F022850F82850E83A37407F0227D017BCD
:1017B500017E00020968D3E53E9400E53D940022D0
:0A17C500D3E53E9400E53D940022B8
:1030BE00E490E6C3F000000090E6C27407F0000052
:0230CE000022DE
:1030390090E6C2E02041054402F0800354FDF0000F
:1030490000002290E6C2E02041054401F0800354CB
:10305900FEF00000002290E6C2E02041054404F0A1
:10306900800354FBF00000002290E6C2E0204005F6
:103079004402F0800354FDF00000002290E6C2E013
:0F3089002040054401F0800354FEF000000022B7
:0F31020090E6C2E02040044404F02254FBF02287
:0A314E00EFF490E6C2F0000000224A
:03319500D29522AE
:10309800D295E4FFFE0FBF00010EBE04F8BFB0F5E5
:0330A800C29522AC
:1025C3008B408A4189428B438A44894512170370A1
:1025D30002054414F9E52312077090E685121701EA
:1025E3007002054414F9EF12077090E68412170184
:1025F3007002054414F9EF120770121703700205F5
:0E2603004414F9ED120770C3E5459542FF221D
:101A93008B408A4189428B438A4489451216487098
:101AA30002054414F9E52312077012164870020563
:101AB3004414F9E522120770121648700205441403
:101AC300F9E5211207701216487002054414F9E56E
:101AD30025120770903F6E121645700205441216C8
:101AE3007F903F6E1216467002054412167F903F98
:101AF3000E1216457002054412167F903F0E121601
:101B0300467002054412167F903F03121645700279
:101B1300054412167F903F031216467002054412C5
:101B2300167F903F051216457002054412167F90EA
:101B33003F051216467002054412167F903F0712A6
:101B430016457002054412167F903F071216467021
:101B530002054412167F903F091216457002054490
:101B630012167F903F091216467002054412167F23
:101B73001216487002054414F9E524120770E4F5BF
:101B830024903F101216467002054412167FE4900B
:101B93003F10F0903F261216467002054412167F3E
:101BA300903F2B1216467002054412167F903F0C8D
:101BB3001216467002054412167F903F0D12164608
:0E1BC3007002054412167FC3E5459542FF22CD
:102F74007F0412314ED2B7D294D207903F19E06049
:082F84000612176912236B22EB
:10284400E5AA20E73A7539017E00121772AD6812C5
:1028540025C3EF2539F539E4F568121772121A9376
:10286400EF2539F5391230F2053990FC00E539F0DD
:10287400FD7C00EC90E69CF0AF05EF90E69DF02225
:06318600EF4480F5682211
:102D2300AD077C01EC7E002400F9EE34F0FA7B0160
:102D33001225C3EF2C90F000F0FB7A00EA90E690A6
:092D4300F0AF03EF90E691F022DD
:102C6D0020072BD207D23EC2007F0512314E7F01C5
:102C7D00122D2312167830E50C12167830E403D29B
:0F2C8D009122D290227B647D017F081200E92200
:10290300203D39D23D1216787003022F747F0412D2
:10291300314ED2B712167820E502D294D20712169E
:102923007830E50C12167830E403D29122D290224B
:0D293300903F19E0600612176912236B2215
:102A2C00EF30E505903F1FEDF0EF30E405903F20CF
:102A3C00EDF0EF30E305903F2AEDF0EF30E205903A
:102A4C003F29EDF0EF30E105903F28EDF0EF30E05D
:072A5C0005903F27EDF02279
:102611008F3F7440C3953F50047F408002AF3FEF2E
:10262100C39418500F7440C3953F50047F408006F7
:10263100AF3F80027F188F3F78407CE77A3F791166
:102641007F0E1217B2784D7CE77A3F79347F0A12F8
:0E26510017B290E74074181216B9E53FF02258
:1017CF008E398F3A8C3B8D3C8A3D8B3E90E6B8E04C
:1017DF0030E70302193D122C3D1217BB402D121793
:1017EF003390E6A0E020E1F9E53E640E453D60034D
:1017FF00021947C2AFAE3DAF3E78117C3F7D017BF2
:10180F00017AE77940120968D2AF22E53C853BF0B7
:10181F0012087F1874000118990002186600441806
:10182F00590049185E004A18560052186D00541896
:10183F00630069189C800018BD800119138002197C
:10184F002DFF01000019470230E1E4FF022D23E4D0
:10185F00FF023186022FE5AF3AAE39022F5AAF3A67
:10186F00AE3902311112167830E503021947E53906
:10187F00453A24FFB39282E53A453970047F0180DF
:10188F00027F00EF24FFB3923F2202247AE4FBFD94
:10189F007F081200E97F007E007D007C0012236B21
:1018AF0012167830E505C290C29122C2912212160B
:1018BF007830E536E539700EC291FBFD7F081200D6
:1018CF00E9C291C29022E539FFBF010812167830A4
:1018DF00E413800CEF6402705FE53AC39480500507
:1018EF00C290D29122C291D29022E539FFBFFF0957
:1018FF00E53AFB7DFF7F088022AC39AD3AE4120355
:10190F00C802236B12167830E52EC3E53994804058
:10191F00047F0980027F0A7B507D020200E9E53ACD
:10192F006006123098D23F22123195C23F22121711
:09193F00BB4005AF3E1226112247
:101DDA008F398D3A8B3B90E6B8E030E703021E6EEE
:101DEA00E53D7074E53E7070E53C7F00FEEF253BF3
:101DFA00FFE43EFEEF8EF012087F1E4000001E45F3
:101E0A0000011E4F01001E4F01011E4F01021E4F0D
:101E1A0001031E4F01041E4F01051E4F01061E4FEE
:101E2A0001071E4F01081E4F01091E4F010A1E58C5
:101E3A00FFFF00001EC4AF39022A63E539FD7C00AA
:101E4A00AF3A022056AB39AD3AAF3B0200E9E53A68
:101E5A006068AD39FF022A2C12174F90E6A0E030D5
:101E6A00E15880F7E53DD39400404F753F01744037
:101E7A00253FF9E434E7FA7B017DFF1225C3EF25FC
:101E8A003FF53F2440F9E434E7FA7B01121A93EF55
:101E9A00253FF53FE53BB4010C1228C4AE3F053F90
:101EAA0012166CEFF090E740E53FF012174FE53A53
:0B1EBA007008E539B401031230F22279
:101FB80090E6B9E01208591FE4101FE4112001400F
:101FC800204DA2204DA32014D42027D5202ED62082
:101FD80033D72038D82040D90000205290E6BAE004
:101FE800FFA3E0FDA3E0FBA3E0F53CA3E0F53DA3E0
:101FF800E0F53E121DDA022054121717C006C0077A
:10200800121694D007D0061217CF8040121717C0A7
:1020180006C007121694D007D006120ED2802D7F64
:1020280001122D23800D122844800812265F800398
:10203800122B06122C3D801490E6BCE024FF92413E
:0E20480012318C8007121CD98002D322C322D1
:100ED2008E398F3A8C3B8D3C8A3D8B3E90E6B8E052
:100EE20030E7030210741217C5400A12173390E656
:100EF200A0E020E1F9E53C853BF012087F0F7B0082
:100F0200010FF400A00FBF00B00F8A00D010230120
:100F1200A0101D01A1101701A2101101A3100B01B5
:100F2200A4100501A50FFF01A60FF901A70FEE01FD
:100F3200B00FE801B10FE201B20FDC01B30FD6012D
:100F4200B40FD001B50FCA01B60FC401B70FB90172
:100F5200D00FB301D10FAD01D20FA701D30FA10161
:100F6200D40F9B01D50F9501D60F8F01D71029FF02
:100F7200001064FF0100001306E490E6C3F00000D5
:100F82000090E6C2E53AF022E53AF5B022E53A13DE
:100F920092B722E53A1392B622E53A1392B522E5C8
:100FA2003A1392B422E53A1392B322E53A1392B27B
:100FB20022E53A1392B122E53A1392B022E53AF5CC
:100FC2009022E53A13929722E53A13929622E53A55
:100FD20013929522E53A13929422E53A13929322C0
:100FE200E53A13929222E53A13929122E53A13924C
:100FF2009022E53AF58022E53A13928722E53A13E8
:10100200928622E53A13928522E53A13928422E5EA
:101012003A13928322E53A13928222E53A1392819D
:1010220022E53A139280221217C55003021306AE2C
:101032003DAF3E7C007D031207A4ED4C600302131A
:1010420006D3E53E9430E53D94004003021306AE1C
:101052003DAF3E783E7C3F7D017B017AE7794002DD
:101062000968E53A6006123098D23F22123195C2E1
:101072003F22E53C853BF012087F12E0000212F9A4
:101082000003120C00A0118400B010FC00D01284E6
:1010920001A0127401A1126401A2125401A312440C
:1010A20001A4123401A5122401A6121401A711FCF5
:1010B20001B011EC01B111DC01B211CC01B311BCD0
:1010C20001B411AC01B5119C01B6118C01B71174B8
:1010D20001D0116401D1115401D2114401D3113450
:1010E20001D4112401D5111401D6110401D712948F
:1010F200FF0012AAFF010000130690E740E5B002CC
:1011020012FF30B7047F0180027F0090E740EF02B8
:1011120012FF30B6047F0180027F0090E740EF02A9
:1011220012FF30B5047F0180027F0090E740EF029A
:1011320012FF30B4047F0180027F0090E740EF028B
:1011420012FF30B3047F0180027F0090E740EF027C
:1011520012FF30B2047F0180027F0090E740EF026D
:1011620012FF30B1047F0180027F0090E740EF025E
:1011720012FF30B0047F0180027F0090E740EF024F
:1011820012FF90E740E5900212FF3097047F018042
:10119200027F0090E740EF0212FF3096047F018049
:1011A200027F0090E740EF0212FF3095047F01803A
:1011B200027F0090E740EF0212FF3094047F01802B
:1011C200027F0090E740EF0212FF3093047F01801C
:1011D200027F0090E740EF0212FF3092047F01800D
:1011E200027F0090E740EF0212FF3091047F0180FE
:1011F200027F0090E740EF0212FF3090047F0180EF
:10120200027F0090E740EF0212FF90E740E5800284
:1012120012FF3087047F0180027F0090E740EF02D7
:1012220012FF3086047F0180027F0090E740EF02C8
:1012320012FF3085047F0180027F0090E740EF02B9
:1012420012FF3084047F0180027F0090E740EF02AA
:1012520012FF3083047F0180027F0090E740EF029B
:1012620012FF3082047F0180027F0090E740EF028C
:1012720012FF3081047F0180027F0090E740EF027D
:1012820012FF3080047F0180027F0090E740EF026E
:1012920012FFAE3DAF3E78407CE77D017B017A3F95
:1012A200793E1209680212F2E4F53F903F241216C9
:1012B20051EFF0903F72121651EFF0121668E56688
:1012C200F0E565121667EFF0C3E53F953EE4953D04
:1012D2005004AF3F8002AF3E90E68BEFF02290E6E3
:1012E200F4E020E1047F0180027F0090E740EFF00C
:1012F20090E68BE53EF02212167890E740F090E6F9
:051302008B7401F022D4
:102C3D00C2AFE4F565F566D2AFC23DD200D2411206
:102C4D003039903F73E02403FF903F72E03400FE73
:102C5D007C007D0A1207A4903F32ECF0A3EDF02228
:0131A4002208
:0F311100AC06C2AFEF903F14F0ECA3F0D2AF22A8
:1014B100AF23E5805403C454F0FEE5B0540F4EF55C
:1014C10023E5236F903F10F0A21B301301B3502589
:1014D100903F31E014F0E07024A21B301301B3728D
:1014E100239223A21B9213A213720B920BA22BA085
:1014F10013922B8000903F2AE0903F31F0A21A30E6
:101501001201B35025903F30E014F0E07024A21A8C
:10151100301201B372229222A21A9212A212720AFC
:10152100920AA22AA012922A8000903F29E0903FBD
:1015310030F0A219301101B35025903F2FE014F083
:10154100E07024A219301101B372219221A21992E3
:1015510011A21172099209A229A011922980009069
:101561003F28E0903F2FF0A218301001B350259092
:101571003F2EE014F0E07024A218301001B3722065
:101581009220A2189210A21072089208A228A0100C
:1015910092288000903F27E0903F2EF0A21D301549
:1015A10001B35025903F23E014F0E07024A21D30D8
:1015B1001501B372259225A21D9215A215720D92E5
:1015C1000DA22DA015922D8000903F20E0903F2389
:1015D100F0A21C301401B35025903F22E014F0E03A
:1015E1007024A21C301401B372249224A21C921400
:1015F100A214720C920CA22CA014922C8000903F89
:101601001FE0903F22F0903F2BE0FF903F26E055F6
:10161100245522FEEF4E903F2BF0903F0DE0FF90BE
:101621003F0CE05524FEE522F45EFEEF4EA3F09060
:101631003F21E0F4552460057F02123186903F215D
:04164100E524F0228A
:10205600EFB40B0040030220E8902066F8282873AE
:1020660002208702208F02209702209F0220A702CB
:1020760020DD0220D20220C70220AF0220B70220B4
:10208600BFEC4D24FF92B7805BEC4D24FF92B580E8
:1020960053EC4D24FF92B6804BEC4D24FF92978073
:1020A60043EC4D24FF9296803BEC4D24FF929180A9
:1020B60033EC4D24FF9293802BEC4D24FF929280BB
:1020C60023EC4D24FF92411230398018EC4D24FF49
:1020D600924112304C800DEC4D24FF924112305F3C
:1020E6008002C322D322EFB40B00400302217E906C
:1020F60020FCF828287302211D02212502212D0229
:10210600213502213D02217302216802215D02214F
:102116004502214D022155EC4D24FF92B7805BEC20
:102126004D24FF92B58053EC4D24FF92B6804BECC4
:102136004D24FF92978043EC4D24FF9296803BEC12
:102146004D24FF92918033EC4D24FF9293802BEC2B
:102156004D24FF92928023EC4D24FF924012307260
:102166008018EC4D24FF9240123085800DEC4D24F2
:0C217600FF92401231028002C322D322EB
:102A6300903F3EE07005EFA2E392B7903F41E070E4
:102A730005EFA2E192B5903F44E07005EFA2E29228
:102A8300B6903F47E07004EF139297903F4AE0708F
:072A930005EFA2E492962278
:1028C400E4FF3097047E0180027E00EE420730B5BB
:1028D400047E0280027E00EE420730B6047E04804D
:1028E400027E00EE420730B7047E0880027E00EECE
:0F28F40042073096047E1080027E00EE420722DB
:1022A300EF14601A14602114602C14603714604218
:1022B3002405704F7FE3123176903F6E80407FE5B7
:1022C300123176903F0E8036C293C2927FEE123166
:1022D30076903F038028C293D2927FEE123176909C
:1022E3003F05801AD293C2927FEE123176903F0758
:1022F300800CD293D2927FEE123176903F09EEF0AA
:04230300A3EFF02232
:1030D000AF6305631222A3E56375F0068485F06390
:0130E00022CD
:102FD000E4F53FE4FBFDAF3F1200E9053FE53FC3E9
:052FE000941040EF22F7
:1000E900AE07C2AF1216C3EFF0121741EBF0EF12D1
:0700F9001686EDF0D2AF22E4
:1026AB00E4FE0567121685E0D394004033E56770AE
:1026BB000E1216C3E0FF7D017C001220EC8021EE90
:1026CB00121741E0656770181216C3E0FFE4FDFCBA
:1026DB001220EC121685E0F46006121685E014F059
:0726EB000EEE641070BE2228
:102EE900E4F5B275B3FF75B5F090E6C3F090E6C2AC
:0D2EF9007407F0C24112304C7FFF022A63C3
:10297D00903F34740A12178630B1047F0180027FB4
:10298D0000EF25E025E04463FF30B0047E018002B6
:10299D007E00EE25E04FF520903F38F0E4A3F0A344
:0C29AD00F0903F3DF0C294C207C291229E
:10265F0090E61274E0F000000090E615F000000024
:10266F0090E611F000000090E610E0547FF00000BB
:10267F000090E613E0547FF000000090E614E05461
:10268F007FF0000000122FE5122FFA90E6837412EC
:0C269F00F07432F090E65CE04402F0229F
:1030F200E4F521F525F524903F2BF0903F0DF022C9
:102BD800903F1F7401F0903F22F0903F20F0903F0B
:102BE80023F0903F2AF0903F31F0903F29F0903F3A
:102BF80030F0903F28F0903F2FF0903F27F0903F23
:032C08002EF02289
:1024CF007F0712314EE4903F72F0A3F0903F70F00F
:1024DF00A3F0D200C23EC23DC207C2B7C297903F1F
:1024EF0011740EF0A37401F0E4A3F0A3F0A3F0A312
:1024FF0004F0E4A3F0A312167730E5047FFF800207
:10250F007F00903F19EF121786A3F0A3F07F01020F
:02251F00314E3B
:102B060012319512317E903F0B7451F0903F2D7427
:102B160001F090E600E054E74410F0903FB412084C
:102B2600184C371B00122A9A1229F312265F122418
:052B36007A43AF01220B
:10218200C3903F32E094015021903F72E0FEA3E001
:10219200FF903F32EEF0A3EFF04E600EC2411230DC
:1021A20039903F327401F0A3E4F0903F13E0602CC9
:1021B200203E13121791EDFFD3E5669FE5659E4021
:1021C2001B122C6D8016121791EEFCE565C313FEEF
:1021D200E56613D39DEE9C4003122903A28092026E
:1021E200A2B09203903F38E520F0E566903F3BF0C5
:1021F200E565A3F0E568C3948040031228441216F3
:102202007830E50A90E6F4E020E003122903303F3B
:05221200031230D02290
:102FE50090E6047480F00000007402F0000000E434
:102FF500F00000002290E6047480F00000007408E0
:0A300500F0000000E4F000000022DB
:1030E1007F007E007D007C0012236B1224CF022919
:0130F1007D61
:10247A001230BEE4F5687F0712314E122FFA122F7E
:10248A00E5903F26743FF0903F0CF0E4903F21F036
:10249A00C23DC2B7C294C207C2911230F2122BD8FF
:1024AA00122FD07D7A12176B12277D122EE9123065
:1024BA00E112167830E5097B507D027F0A1200E9A5
:0524CA007F0102314E0C
:102A9A00E4F53912170E7D087FF87E1D122573E4BE
:102AAA00F5397440253912166FE0FDE53975F002E3
:102ABA00A42474F9740135F08982F583EDF005399F
:062ACA00E539B408DD222D
:1023CC008B398A3A893BE4F53C1230248F3DE53D4C
:1023DC0025E02402900192F0E4F53CAF3DEF3395FB
:1023EC00E0FEC3E53C9FEE6480F87480985027AB08
:1023FC0039AA3AA93B853C82758300120743FDE557
:10240C003C75F002A42494F9740135F08982F583AB
:07241C00EDF0053C80C52234
:1029F30012170E7D017F037E0012257390E740E0DE
:102A030090010CF090E740E0247F600B0470107B92
:102A1300FF7A2D794C800E7BFF7A2D795A80067BC5
:092A2300FF7A2D79671223CC2201
:0E312000903F137401121677700312300F22C5
:102F5A00EF4E60047F0180027F00903F13EFF07014
:0A2F6A0008121678700312312E22AF
:1029B9001226AB1214B1D56430903F73E004F07065
:1029C90006903F72E004F0C3903F73E0940A903F91
:1029D90072E094004010C2AF0566E56670020565B5
:0A29E900D2AFE4F0A3F0756464229D
:10300F007B807DFF7F031200E9D297C24112304CC3
:05301F00C24102305F18
:0B312E00C2977B80E4FD7F030200E9F4
:102DC000C0E0C083C082C085C084C086758600D242
:102DD0003A1216ED7401F0D086D084D085D082D01E
:042DE00083D0E0328A
:102E6F00C0E0C083C082C085C084C0861216EA74D9
:102E7F0004F0D086D084D085D082D083D0E032C009
:102E8F00E0C083C082C085C084C0861216EA740277
:0E2E9F00F0D086D084D085D082D083D0E032AF
:102B7000C0E0C083C082C085C084C08675860085E1
:102B8000100C85110D12179C85080E85090F121760
:102B9000A71216ED7410F0D086D084D085D082D0E4
:042BA00083D0E032CC
:102DE400C0E0C083C082C085C084C086758600D21E
:102DF4003C1216ED7408F0D086D084D085D082D0F1
:042E040083D0E03265
:101EC500C0E0C083C082C085C084C086758600908E
:101ED500E680E030E71285080C85090D12179C8510
:101EE500100E85110F1217A71216ED7420F0D0866B
:0B1EF500D084D085D082D083D0E032B2
:1031A50032323232323232323232323232323232FA
:1031B50032323232323232323232323232323232EA
:0431C500323232323E
:1027C100AB07AA06AC05E4FD903F2DE0600B7E004F
:1027D1000DEE24BB12177EEAF0AE050D74BB2E126E
:1027E100177EEBF0AF050D74BB2F12177EECF09046
:1027F1003F0BE0FF7A3F7BBB122F22903F0BE0FFA4
:03280100022AD0D8
:102B3B008E418F428D438A448B45E4F546E546C36F
:102B4B00954350200542E542AE417002054114FF0A
:102B5B00E5452546F582E43544F583E0FD1227C1B2
:052B6B00054680D9229F
:102573008E418F428D438A448B45E4FDF546903F5F
:102583002DE06012E541FF7E000DEE24BBF582E4F1
:10259300343FF583EFF0AE050D74BB2EF582E434C2
:1025A3003FF583E542F0903F0BE0FF7A3F7BBB12A0
:1025B3002F22903F0BE0FFAB45AA44AD43022F0609
:02319800D32240
:102EAD0000000090E6247402F0000000E490E62596
:0E2EBD00F000000090E6BAE0903F2CF0D32227
:10315800903F2C1216B504F0D32290E6BAE0903FC7
:0E31680002F0D322903F021216B504F0D322DB
:0A319A00D322D322D322D322D32262
:101CD90090E6BAE0753900F53AA3E0FEEE42399094
:101CE900E6BEE0753B00F53CA3E0FEEE423B90E624
:101CF900B8E064C06003021D80E53C453B70030207
:101D09001DD990E6A0E020E1F9C3E53C9440E53B0C
:101D190094005008853B3D853C3E8006753D007525
:101D29003E4090E6B9E0B4A31EE4F53FF540121732
:101D390029503812175CE0FF1216F4EFF00540E560
:101D49004070EB053F80E7E4F53FF5401217295055
:101D5900101216F474CDF00540E54070EF053F8090
:101D6900EB12170CAF3AAE391225731216BAE53ECB
:101D7900F01216D2021D0290E6B8E064407051E5F7
:101D89003C453B604B1216BAF090E6A0E020E1F921
:101D990090E68BE0753D00F53E90E6B9E0B4A31EF0
:101DA900E4F53FF540121729501E1216F4E0FF1210
:101DB900175CEFF00540E54070EB053F80E712172F
:101DC9000CAF3AAE39122B3BE53E1216D2021D88F2
:011DD90022E7
:03004300021F0099
:03005300021F0089
:101F0000022DC000022E8E00022E6F00022DE40072
:101F1000022B7000021EC5000231A5000231A6008E
:101F20000231A7000231A8000231A9000231AA0043
:101F30000231AB000231AC000231AD000231AE0023
:101F40000231AF000231A6000231B0000231B1000F
:101F50000231B2000231B3000231B4000231B500E7
:101F60000231B6000231A6000231A6000231A600FD
:101F70000231B7000231B8000231B9000231BA00B3
:101F80000231BB000231BC000231BD000231BE0093
:101F90000231BF000231C0000231C1000231C20073
:101FA0000231C3000231C4000231C5000231C60053
:081FB0000231C7000231C80034
:102E08008F7D903FBAEDF07A3F7BBA7D01122F2279
:102E18007A3F7BB87D02AF7D122F06903FB8E0FE67
:042E2800A3E0FF2202
:10294000AE07C2E990E678E04480F0EE25E090E63C
:1029500079F090E678E030E0F9ED90E679F090E6F5
:1029600078E030E0F990E678E04440F090E678E0F6
:0D29700030E0F990E678E020E6F9D2E922A7
:102FA300AC071229407A3F7BBB7D02122F06903F6C
:072FB300BBE0FEA3E0FF22DA
:08317600AD077F40122FA322D8
:102CCB0090E682E030E004E020E60B90E682E03014
:102CDB00E119E030E71590E680E04401F07F147EC7
:0C2CEB00001226F290E680E054FEF02279
:102D9B0090E682E044C0F090E681F04387010000AA
:042DAB000000002202
:102C9C0030410990E680E0440AF0800790E680E03D
:102CAC004408F07FDC7E051226F290E65D74FFF09E
:0F2CBC0090E65FF05391EF90E680E054F7F0223E
:08317E00E4F56ED2E9D2AF22A4
:102AD00090E678E020E6F9C2E990E678E04480F0FC
:102AE000EF25E090E679F090E678E030E0F990E6C6
:102AF00078E04440F090E678E020E6F990E678E06F
:062B000030E1D6D2E9220B
:102C0B00A90790E678E020E6F9E56E702390E67868
:102C1B00E04480F0E925E090E679F08D69AF03A9F7
:102C2B0007756A018A6B896CE4F56D756E01D322A9
:022C3B00C322B2
:102BA400A90790E678E020E6F9E56E702590E678CE
:102BB400E04480F0E925E0440190E679F08D69AFC6
:102BC40003A907756A018A6B896CE4F56D756E0358
:042BD400D322C32223
:03004B00021BD1C4
:101BD100C0E0C083C082C085C084C086758600C055
:101BE100D075D000C000C001C002C003C006C0074C
:101BF10090E678E030E206756E06021CBB90E6784E
:101C0100E020E10CE56E64026006756E07021CBB04
:101C1100E56E24FE605F14603624FE7003021CAC86
:101C210024FC7003021CB824086003021CBBAB6ACD
:101C3100AA6BA96CAF6D056D8F8275830012074386
:101C410090E679F0E56D65697070756E05806B9051
:101C5100E679E0AB6AAA6BA96CAE6D8E82758300E2
:101C6100120782756E02E5696401704E90E678E0B4
:101C71004420F08045E56924FEB56D0790E678E0E3
:101C81004420F0E56914B56D0A90E678E04440F02F
:101C9100756E0090E679E0AB6AAA6BA96CAE6D8EA9
:101CA10082758300120782056D800F90E678E0440B
:101CB10040F0756E008003756E005391DFD007D040
:101CC10006D003D002D001D000D0D0D086D084D0AD
:081CD10085D082D083D0E032FF
:102CF700A907AE14AF158F828E83A3E06403701704
:102D0700AD0119ED7001228F828E83E07C002FFDCB
:0C2D1700EC3EFEAF0580DF7E007F002256
:102F0600122BA4E56E24FA600E146006240770F3F3
:102F1600D322E4F56ED322E4F56ED322122C0BE510
:102F26006E24FA600E146006240770F3D322E4F5CB
:082F36006ED322E4F56ED322F4
:1026F2008E398F3A90E600E054187012E53A2401C0
:10270200FFE43539C313F539EF13F53A801590E636
:1027120000E05418FFBF100BE53A25E0F53AE53921
:1027220033F539E53A153AAE39700215394E60057E
:06273200122DAF80EE2223
:102DAF007400F58690FDA57C05A3E582458370F937
:012DBF0022F1
:0B313900253032625800253034580069
:022FA000C1422C
:102E2C007B017A3F797422743FF59A7474F59B7424
:102E3C00E7F59D74C0F59EE42290E67BE090E67C7D
:022E4C00F02272
:05318C00A24192422265
:10273800204204E4FEFF2290E6A2E020E1F9122EF6
:102748002C123024EF2401F57AE43EF579122E3369
:10275800FFFEC3EF957AE5796480F8EE64809850BF
:102768000A122E450FBF00010E80E7E57A90E68F2A
:05277800F0AE79FF2224
:10242300204204E4FEFF22E5AA20E7FB122E2C1231
:102433003024EF2401F57CE43EF57B743FF59A7478
:1024430074F59B74FCF59D7400F59EE4FFFEC3EFE9
:10245300957CE57B6480F8EE648098500A122E45E3
:102463000FBF00010E80E7E57B90E69CF0E57C90D2
:07247300E69DF0AE7BFF22A5
:102884008B748A758976204204E4FEFF221228BAEA
:102894008E1C8F1D85741985751A85761B122E2C36
:1028A4001225211228BA74742FF582743F3EF583E1
:1028B400E4F012273822AB74AA75A97612302422C8
:1030AB00204204E4FEFF22903F74EFF0E4A3F01201
:0330BB0027382291
:102F3E00204204E4FEFF22754AFF754B31754C3971
:0C2F4E008F4D122E2C120ABF12273822C1
:102ECB00204204E4FEFF22754AFF754B31754C3FDF
:0E2EDB008E4D8F4E122E2C120ABF1227382257
:1023070090E685E02405F56F204204E4FEFF22787D
:10231700747C3F7D01120A4690E6A2E030E1079007
:10232700E685E0B56FF2122E2C123024EF2401F56A
:1023370073E43EF572122E33F570F571C3E57195AE
:1023470073E5726480F8E570648098500D122E452D
:102357000571E57170E6057080E2E57390E68FF030
:04236700AE72FF2231
:1001B20002046DE86480F8E933E83360110460F00A
:1001C200ED33EC337009E8FCE9FDEAFEEBFF2204B3
:1001D20060DED3EB9FEA9EE99DE8C2E78CF0C2F7AE
:1001E20095F0400CE8CCF8E9CDF9EACEFAEBCFFB7A
:1001F20012043885D0F05804700320D5B3E8047097
:10020200075002B2D502047792D5EC0460F7E4CC31
:10021200C0E0C398F8603B94186008400DD0E0FB42
:1002220002044FE4FBFAC9FC8028E830E406E4C982
:10023200FBE4CAFCE830E305E4C9CACBFCE8540796
:100242006010F8C3E913F9EA13FAEB13FBEC13FCA1
:10025200D8F130F52FC3E49CFCEF9BFFEE9AFEED44
:1002620099FDD0E0FBEF4E4D4C701222DB030204ED
:1002720074EC2CFCEF33FFEE33FEED33FDED30E793
:10028200EB02044FEF2BFFEE3AFEED39FDD0E0FB1F
:1002920050130BBB0003020477ED13FDEE13FEEFC8
:1002A20013FFEC13FC02044F020477EC5D046005BB
:1002B200E85904700302046D120438580460F6EC25
:1002C2004860F2EC7004FDFEFF22C860DB2481C8A6
:1002D2005009C398600250060204749850CAF5820D
:1002E200E9294B4A7005AB8202046375F0007C1A5F
:1002F2007880C3EF9BEE9AED99400DC3EF9BFFEE22
:100302009AFEED99FDE842F0DC23ACF0D0E0FFD09C
:10031200E0FED0E0FDAB8220E7101BEB60BAEC2CD4
:10032200FCEF33FFEE33FEED33FD02044FE803F83A
:1003320030E705C0F075F000EF2FFFEE33FEED332E
:10034200FD40B830E7C280AA74F8CC6480CCC8649F
:1003520080C8F58204604FC3EB9FF5F0EA9E42F03D
:10036200E99D42F0E89C45F0603C501DE5825FFF4C
:10037200E582D313CB5BCBF42B5582FB50280ABA10
:10038200002409B9002008801DE5825BFBE582D3C9
:1003920013CF5FCFF4C3132F5582FF50090EBE0057
:1003A200050DBD00010CC3EB9FF5F0EA9E42F0E99A
:1003B2009D42F0E89C45F06007CC4820E701B3EC91
:1003C2002275F020800E75F010800575F0087D0012
:1003D2007E007F003392D530D5031207F9EC33400B
:1003E20010EF33FFEE33FEED33FDEC33FCD5F0EDD1
:1003F20022E5F0247EA2D513CC92E7CDCEFF22EDEA
:10040200D2E7CD33EC3392D524814006E4FFFEFDE2
:10041200FC22FCE4CFCECDCC24E0501174FF80ED61
:10042200C3CC13CCCD13CDCE13CECF13CF0470F0EB
:0604320030D5DE0207F9DF
:100A6300E55E244AF8E6055E227847303702784A85
:100A7300E475F00112084902072A2030EB7F2ED2D9
:100A8300308018EF540F2490D43440D4FF30340B0B
:100A9300EF24BFB41A0050032461FFE55F60021521
:100AA3005F0562E5627002056130370D7847E475D2
:100AB300F001120849EF020770022D747403D23754
:100AC3008003E4C237F55E8B478A488949E4F55FC2
:100AD300F561F562E55F60077F20120A9E80F57578
:100AE30060FFC231C230C232C233C235C236C238ED
:100AF300120A6CFF700D3037057F00120AAFAF6228
:100B0300AE6122B4255FC2D5C234120A6CFF24D071
:100B1300B40A00501A75F00A785F30D50508B6FF9D
:100B23000106C6A426F620D5047002D23380D92448
:100B3300CFB41A00EF5004C2E5D234020D9CD23177
:100B430080C6D23080C0D23280BCD2D580BAD235F2
:100B530080B47F20120A9E2032077401B55F0040E3
:100B6300F1120A63FF120A9E020AD7D238D23680E4
:100B730095120A63FB120A63FA120A63F94A4B706D
:100B83000679937A0E7BFF20322EE55F602A7E0082
:100B93008E8275830012074360060EEE656070F067
:100BA300C2D5EBC0E0EAC0E0E9C0E0EE120DFCD034
:100BB300E0F9D0E0FAD0E0FB12072AFF60AAEBC00D
:100BC300E0EAC0E0E9C0E0120A9ED0E02401F9D0D7
:100BD300E03400FAD0E0FBE5600460DCD560D98046
:100BE30087D23280A2120DDF60F7E5607001041234
:100BF3000482A960600DE560600914F560120E8639
:100C0300EF60F3EA30E702F404C3995077EAF4257E
:100C1300600430E701E404F560800D120DDF60C16C
:100C2300EA05602560120482EA785DF630E701E4A4
:100C3300256004D5600420350114120DFCE4C0E0E6
:100C4300120E86785DE6601320E70714F6120A8613
:100C5300802204F6D0E014C0E07F00120A86E5602B
:100C63006007120A7D1560800B303503120A7DD0B0
:100C7300E0020AD7D0E00480C5120DDF60A0E56072
:100C830004120482785DEAF6E5602035026001040F
:100C93002404120DFC74FF04C0E0120E86120A86AF
:100CA300E5602035026003120A7DD0E0B560E87F7D
:100CB30045120A90785DE67F2B30E7047F2DF4041C
:100CC300C0E0120A9ED0E075F00A84C0F0120A87D1
:100CD300D0E0120A87020AD7791080027908C23657
:100CE300C2388008D2D5790A8004790AC2D5E56072
:100CF300047002F560E4FAFDFEFF120A63FC7B0850
:100D0300203113120A63FD7B1030300A120A63FE8E
:100D1300120A63FF7B20EC3382D592D55013C3E4D0
:100D23003030069FFFE49EFEE42031039DFDE49CEA
:100D3300FCE4CBF8C231EC700CCFCECDCCE824F878
:100D4300F870F38017C3EF33FFEE33FEED33FDECA2
:100D530033FCEB33FB994002FB0FD8E9EB30310551
:100D6300F8D0E0C448B231C0E00AEC4D4E4F7820D1
:100D73007B0070C2EAB5600040BCC0E0120DFED03B
:100D8300F0D0E0203104C4C0E0C4B231C0F0120A94
:100D930087D0F0D5F0EB020AD71208590B74530C25
:100DA300DB580B454C0B41420CDF4F0CE7440CE77F
:100DB300490B5A430CED550C1E460C7C450BE8477A
:100DC3000EB3500B492D0B4D2E0B702B0B51230BD8
:100DD3006E200E9C2A0B094800000B68E560B4FFE7
:100DE30003756006120A63FC120A63FD120A63FEAE
:100DF300120A63FF78560204B1790AA2D52033148C
:100E0300303509B910020404B9080104A2D520360B
:100E1300025001042032689232B55F005034C0E0C2
:100E23007F203033197F30A23272367235500F1261
:100E33000E55C232C236C235C2387F30800F3035CC
:100E430003E9C0E0120A9E303503D0E0F9D0E0B5E3
:100E53005FCC3035177F30B9100C120A9E7F5830A3
:100E630034077F788003B90803120A9E3032057F66
:100E73002D020A9E7F202038F87F2B2036F3229202
:100E83003280CF7F00B4070050052456F8E6FF22D6
:100E9300286E756C6C2900D231120A633031F8C2A6
:100EA30031785F30D50108F6020B092D50434958BC
:100EB300120A632403B405004001E4900EAE9312BA
:0F0EC3000A8F743A120A8FD233755F04020CDB68
:10043800E9D2E7C933E833F892D5EDD2E7CD33EC0A
:1004480033FC5002B2D522EC30E7100FBF000C0E7F
:10045800BE00080DBD00040BEB6014A2D5EB13FC25
:10046800ED92E7FD2274FFFCFDFEFF22E480F8A276
:10047800D574FF13FC7D80E480EFF920E72824F988
:1004880050037907E4F42402FB18DBFDE624FB5053
:1004980014E9600DE4F618E604F6B40A08E4F6D99F
:1004A800F57401F60A22C2D522ED33EC3392D5FA5F
:1004B800602AB4FF33EDC2E77BFF60067A0479D681
:1004C800E4227A0479DF20D5047A0479DA224E61AD
:1004D8004E002B494E46002D494E4600E47A08F658
:1004E80008DAFC7B00740722E8C0E0ECC0E0EDC04D
:1004F800E0EEC0E0EFC0E0EA75F010A4CAABF0751A
:10050800F04DA42BFBE435F0FCEA2410FAEB34C5DB
:10051800FBEC34D9FCEDC2E7FF75F056A4F42411C6
:10052800C5F0F434C58FF0A42AE5F03BE43CF6208E
:10053800E7141206EAD0E0FFD0E0FED0E0FDD0E0FC
:10054800FC1202AD8014F4041206EAD0E0FFD0E0F9
:10055800FED0E0FDD0E0FC1205B4D0E0F8E6FAEDFC
:10056800D2E7CD33EC332482FBE4C3CF33CFCE3391
:10057800CECD33CD33DBF37B0775F00A846004F608
:10058800081B0AE5F0F6088FF0740AA4FFACF08E99
:10059800F0740AA42CFEACF050010C8DF0740AA47F
:1005A8002CFDE435F0F608DBDE740722EC4D601113
:1005B800E8497017ED33EC3304600DE4FCFFFEFDF1
:1005C80022E933E8330470F802046D120438580441
:1005D8006009E4CC24815006285009020477284099
:1005E80003020474C0E0EB4A7044B98006D0E0FB13
:1005F800020463EF4E701CBD8008EBFFEAFEE9FDC4
:1006080080EBE98DF0A4FEE5F002069DE9CDF9EA5C
:10061800FEEBFFEF89F0A4FCE5F0CE89F0A42EFFF5
:10062800E435F0CD89F0A42DFEE435F08067EF4E77
:100638007005BD80D780C3EF8BF0A4ACF0EE8BF0D3
:10064800A42CFCE435F0F8EF8AF0A42CE5F038FC93
:10065800E433CB8DF0A42CFCE5F03BF8EE8AF0A453
:100668002CFCE5F038F8E433CF89F0A42CFCE5F055
:1006780038CF3400CE89F0A42FFFE5F03EFEE433F6
:10068800C98DF0A42EFEE5F039CD8AF0A42FFFE540
:10069800F03EFEE43DFD33D0E0FB50070BBB000FFE
:1006A800020477EC2CFCEF33FFEE33FEED33FD0252
:1006B800044F3F8000004120000042C80000447AF7
:1006C8000000461C400047C35000497424004B18E2
:1006D80096804CBEBC205A0E1BCA6753C21C749D20
:1006E800C5AEFB60065407601C2323120718EB54A1
:1006F8003860091207041207131205B4ECF8EDF973
:10070800EEFAEFCB22EB12071380F1543803241CC6
:100718009006BAFE93FC0EEE93FD0EEE930ECE936A
:02072800FF22AE
:03000000022217C2
:0C221700787FE4F6D8FD75817D02225E20
:10072A00BB010689828A83E0225002E722BBFE02CD
:10073A00E32289828A83E49322BB010CE58229F5AC
:10074A0082E5833AF583E0225006E92582F8E6221B
:10075A00BBFE06E92582F8E222E58229F582E583D5
:10076A003AF583E49322BB010689828A83F02250F8
:10077A0002F722BBFE01F322F8BB010DE58229F53F
:10078A0082E5833AF583E8F0225006E92582C8F625
:10079A0022BBFE05E92582C8F222BC000BBE002955
:1007AA00EF8DF084FFADF022E4CCF875F008EF2F5E
:1007BA00FFEE33FEEC33FCEE9DEC984005FCEE9D1B
:1007CA00FE0FD5F0E9E4CEFD22EDF8F5F0EE842037
:1007DA00D21CFEADF075F008EF2FFFED33FD400798
:1007EA00985006D5F0F222C398FD0FD5F0EA22C33D
:1007FA00E49FFFE49EFEE49DFDE49CFC22EB9FF552
:10080A00F0EA9E42F0E99D42F0E89C45F022A88277
:10081A008583F0D083D08212082F12082F12082F56
:10082A0012082FE473E493A3C583C5F0C583C8C532
:10083A0082C8F0A3C583C5F0C583C8C582C822FA99
:10084A00E6FB0808E6F925F0F618E6CA3AF622D0D9
:10085A0083D082F8E4937012740193700DA3A3936A
:10086A00F8740193F5828883E4737402936860EFE5
:10087A00A3A3A380DFD083D082F8E493701274011B
:10088A0093700DA3A393F8740193F5828883E4739C
:10089A00740293B5F0067403936860E9A3A3A3A353
:0208AA0080D8F4
:102D7400EFB40A07740D122D7F740A309811A899C4
:102D8400B8130CC2983098FDA899C298B811F630BF
:072D940099FDC299F5992297
:102521008B168A178918E4F51EF51FE51D151DAEDA
:102531001C7002151C4E6033AB19AA1AA91B120795
:102541002AFFAB16AA17A918051FE51FAC1E7002BA
:10255100051E14F5828C83EF120782EF60CD7401A2
:10256100251BF51BE4351AF51A80C0AB16AA17A96D
:0225710018222E
:10302400E4FFFE12072A600C0FEF70010E09E9702D
:05303400F20A80EF220A
:1008AC00E709F608DFFA8046E709F208DFFA803E2E
:1008BC0088828C83E709F0A3DFFA8032E309F6081B
:1008CC00DFFA806EE309F208DFFA806688828C8397
:1008DC00E309F0A3DFFA805A89828A83E0A3F60841
:1008EC00DFFA804E89828A83E0A3F208DFFA804225
:1008FC0080D280FA80C680D4805580F28029801006
:10090C0080A680EA809A80A880DA80E280CA80295A
:10091C0088848C8589828A83E493A30586F0A30559
:10092C0086DFF5DEF3800B89828A83E493A3F608D5
:10093C00DFF9ECFAA9F0EDFB2288848C8589828A98
:10094C0083E0A30586F0A30586DFF6DEF480E38959
:10095C00828A83E493A3F208DFF980D688F0EF60F3
:10096C00010E4E60CD88F0ED2402B4040050C3F5A6
:10097C0082EB2402B4040050B9232345822390084F
:10098C00FC73E709F60870FA8046E709F20870FA7A
:10099C00803E88828C83E709F0A370FA8074E309A7
:1009AC00F60870FA806CE309F20870FA80648882A9
:1009BC008C83E309F0A370FA805889828A83E0A3C0
:1009CC00F60870FA804C89828A83E0A3F20870FAE8
:1009DC00804080D280FA80C680D4805180F28027FB
:1009EC00801080A680EA809A80A880DA80E280CA93
:1009FC00802788848C8589828A83E493A30586F07A
:100A0C00A3058670F5800B89828A83E493A3F6088C
:100A1C0070F9ECFAA9F0EDFB2288848C8589828A26
:100A2C0083E0A30586F0A3058670F680E589828AAB
:100A3C0083E493A3F20870F980D888F0ED2402B413
:100A4C00040050CEF582EB2402B4040050C42323DE
:070A5C004582239009DE73BF
:10222300021948E493A3F8E493A34003F68001F270
:1022330008DFF48029E493A3F85407240CC8C333BC
:10224300C4540F4420C8834004F456800146F6DF8B
:10225300E4800B0102040810204080902F8CE47E60
:10226300019360BCA3FF543F30E509541FFEE49380
:10227300A360010ECF54C025E060A840B8E493A347
:10228300FAE493A3F8E493A3C8C582C8CAC583CA72
:10229300F0A3C8C582C8CAC583CADFE9DEE780BE2A
:012FA200002E
:00000001FF
